S123D8008E00FF8600B710268601B740008630B7102B860CB7102D86A097028600970A86EC
S123D820FF9711BDD9DABDD8BF86009709CE02BCBDD8BBBDD9E281A0270D7C000927E7CE49
S123D84002BCBDD8BB20EC18CE0003BDD97B9611270718CE0003BDDA0FB6102E842027404D
S123D860B6102F813F2611960A8101263318CE0003C606BDDA7420B1814326068600970A95
S123D880201E815226068601970A2026812B260686FF9711201C812D26068600971120125E
S123D8A0960A8100260C18CE0002C607BDDA747ED829CE02BCBDD8BB7ED8290926FD39C64C
S123D8C010F71000C630F71000010101C610F71000010101C600F71000C610F710000101A1
S123D8E001C600F71000C610F71000010101C600F71000C610F71000010101C600F71000FC
S123D900C610F71000C610F71000CE0962BDD8BBC630F71000CE02F0BDD8BB860797011876
S123D920CED9748608970018A600482411C630F71000C620F71000C630F71000200FC6107C
S123D940F71000C600F71000C610F710000101017A000026D5CE001EBDD8BB18087A0001C3
S123D96026C1CE0128BDD8BBC610F71000CE4E20BDD8BB3906C1080002FF01BDD9E218A7CB
S123D980001808CE001EBDD8BBBDD9E218A7001808CE001EBDD8BBBDD9E218A7001808CE6F
S123D9A0001EBDD8BBBDD9E218A7001808CE001EBDD8BBBDD9E218A7001808CE001EBDD88A
S123D9C0BBBDD9E218A700CE001EBDD8BBBDD9E2CE001EBDD8BBBDD9E239CC0000DD0BDD1F
S123D9E00D39C610F71000C630F71000010101C610F710008608970048F61000C4011BC60A
S123DA0000F71000C610F710007A000026EA3918A6052603BDD9DA4F18E6002A0143DD0F58
S123DA20930B1A8300022F07DC0F830002DD0BDC0B930F1A8300022F07DC0FC30002DD0B21
S123DA404F18E6012A0143DD0F930D1A8300022F07DC0F830002DD0DDC0D930F1A83000221
S123DA602F07DC0FC30002DD0D960C18A700960E18A70139B6102E848027F918A600B71037
S10ADA802F18085A26EE39A5
S9030000FC
